:020000040000FA
:0600000040EF07F01200C2
:0608000040EF07F01200BA
:06082A0001009E0E00001B
:08083000000200002700000097
:08083800D9CFE6FFE1CFD9FFA3
:10084000040EE126DE6ADE6ADE6ADD6ADD52DD5212
:10085000FD0EDBCF00F0FE0EDBCF01F0026A036A73
:1008600001AE02D002680368D9CFE9FFDACFEAFF10
:10087000030EEB500318E8AE02D0033408D000504A
:10088000EE5C0150EE580250EE580350EE580FE265
:100890000C0EE66E20EC07F0E552D9CFE9FFDACF77
:1008A000EAFFEE2A000EEE22EE22EE22D1D7040E4F
:1008B000E15C02E2E16AE552E16EE552E7CFD9FF81
:1008C00012000F0EC16E070EB46E936A300E926E58
:1008D0000F0E946EF19E1200D9CFE6FFE1CFD9FF43
:1008E000020EE1268250020B01E0010E080DF3CF4B
:1008F00002F08250010B040DF3CF01F08050200B69
:1009000001E0010EE824006E8050100B01E0010EA2
:10091000002401240224DE6EDD6ADECF00F0DDCF8C
:1009200001F000C0F3FF01C0F4FF020EE15C03E23E
:1009300000D0E16AE552E16EE552E7CFD9FF12003F
:100940008092010EE66EE66A77DFE552E55280841A
:10095000010EE66EE66A70DFE552E5528094010E04
:10096000E66EE66A69DFE552E55212008082010E0A
:10097000E66EE66A61DFE552E5528084010EE66EBE
:10098000E66A5ADFE552E5528094010EE66EE66AA9
:1009900053DFE552E5521200380E816ED1DF320E80
:1009A000E66EE66A49DFE552E552010E816EC8DF68
:1009B000320EE66EE66A40DFE552E5520D0E816EBC
:1009C000BFDF320EE66EE66A37DFE552E552060E0D
:1009D000816EB6DF320EE66EE66A2EDFE552E55234
:1009E0001200010E816EACDF0A0EE66EE66A24DFAD
:1009F000E552E5521200D9CFE6FFE1CFD9FF020E52
:100A0000816E9EDF0A0EE66EE66A16DFE552E5525B
:100A1000FD0EDBCFE6FFFE0EDB50280DF350E55256
:100A2000E724E76EFE0EE7CFDBFFFD0EDB6AFE0E6E
:100A3000DB50F36EFD0EDBCFF4FFF350F45C0CE201
:100A4000140E816E7DDF010EE66EE66AF5DEE5527C
:100A5000E552FD0EDB2AEBD7E552E7CFD9FF1200B6
:100A6000D9CFE6FFE1CFD9FFFE0EDB50816E7EDFEE
:100A7000010EE66EE66AE0DEE552E552E552E7CFAA
:100A8000D9FF1200D9CFE6FFE1CFD9FFFD0EDBCFB2
:100A9000E9FFFE0EDBCFEAFFEF500EE0FD0EDBCFED
:100AA000E9FFDB2AFE0EDBCFEAFF01E3DB2AEF5092
:100AB000E66ED6DFE552EAD7E552E7CFD9FF12005E
:100AC00002012B6B300E926EF00E936EEF0E276FBD
:100AD00027C281FF040E286F2851000821E2275108
:100AE000FE0BE842276F27C281FF050EE66EE66A1D
:100AF000A3DEE552E5528150100B09E08150200B36
:100B000006E08150400B03E08150800B01E10AD8E0
:100B100002012B0502E12C5104D02805286FDCD7F7
:100B2000CFD71200F00E936E81CF2AF202012A1560
:100B3000296F0F0E2715276F27512911276F81CF96
:100B40002AF2F00E2A15296FF00E295D01E0F7D781
:100B5000936A06D82DC22CF20201010E2B6F1200EF
:100B600002012E6B100E2E5D14E22E51EA6A000F68
:100B7000E96E020EEA22EF50275D08E12E51EA6A83
:100B8000100FE96E020EEA22EFCF2DF22E292E6F02
:100B9000E9D72DC281FF640EE66EE66A4DDEE552AE
:100BA000E552120002012F6B070E2F5D1DE288DF58
:100BB0000201306F2F51EA6A310FE96E020EEA220C
:100BC00030C2EFFF2F51EA6A310FE96E020EEA22BE
:100BD000EF50460802E108D004D030C2E6FF40DF03
:100BE000E55202012F2BE0D72F51EA6A310FE96E4F
:100BF000020EEA22EF6A120002012F6B070E2F5D30
:100C000016E22F51EA6A310FE96E020EEA22EF5026
:100C1000E66E26DFE55202012F29EA6A310FE96EFE
:100C2000020EEA22EF5001E102D02F2BE7D712008B
:100C3000D9CFE6FFE1CFD9FFE652F250800B01E0B9
:100C4000010EDF6EF29EA69EA69CA684FE0EDB50D1
:100C5000A96EFD0EDB50A86E550EA76EAA0EA76EEC
:100C6000A682A6B2FED7A694DF50E8B0F28EE8A026
:100C7000F29EE552E552E7CFD9FF1200D9CFE6FF49
:100C8000E1CFD9FFA69CA69EFE0EDB50A96EA680E2
:100C9000A85000D0E552E7CFD9FF120012DE320E85
:100CA000E66EE66AC9DDE552E55276DE9ADEE66A70
:100CB000E66AA1DEE552E552200EE66E020EE66E11
:100CC000E1DEE552E552E66A010EE66E94DEE5529B
:100CD000E552E66AD3DFE55202013A6F010EE66E95
:100CE000CDDFE55202013B6F3AC2E6FFB9DEE552C5
:100CF0003BC2E6FFB5DEE552E80EE66E030EE66E99
:100D00009BDDE552E5526DDE3E0EE66EA9DEE55254
:100D1000D7DE0201306F430E305D08E1200EE66E33
:100D2000020EE66EAFDEE552E55201D0F1D7E66A7B
:100D3000010EE66E60DEE552E552C2DE02013A6F58
:100D40003AC2E6FF8DDEE552BBDE02013B6F3BC2DD
:100D5000E6FF86DEE5523AC2E6FFE66A69DFE55263
:100D6000E5523BC2E6FF010EE66E62DFE552E55258
:100D7000E66A84DFE55202013A6F010EE66E7EDF1D
:100D8000E55202013B6F2A0EE66E6ADEE5523AC278
:100D9000E6FF66DEE5523BC2E6FF62DEE552FFD7C4
:020DA00012003F
:0E0DA2002A0EF66E080EF76E000EF86E0001B7
:100DB0000900F550656F0900F550666F03E165673E
:100DC00001D03DD00900F550606F0900F550616F0A
:100DD0000900F550626F09000900F550E96E09003D
:100DE000F550EA6E090009000900F550636F09002B
:100DF000F550646F09000900F6CF67F0F7CF68F08F
:100E0000F8CF69F060C0F6FF61C0F7FF62C0F8FF7D
:100E10000001635302E1645307E00900F550EE6EF0
:100E20006307F8E26407F9D767C0F6FF68C0F7FF09
:100E300069C0F8FF00016507000E665BBFD71200AE
:100E4000FF0EE350066E480E01D04C0EE76EE72E03
:100E5000FED7E76AE72EFED7062EF7D7000012006E
:100E6000000EF36E00EE00F0080E01D81200EA60EA
:100E700002D0EE6AFCD7F350E9601200EE6AFCD7AC
:100E800012EE40F022EE40F0F86A059CD1EC06F03C
:0C0E90004EEC07F04EEC06F0FBD7120011
:020E9C00120042
:020E9E00EEED77
:100EA000EBE7DEDDDBD7BEBDBBB77E7D7B773031C8
:100EB0003233343536373839414243444546434C62
:050EC0004156453A0017
:00000001FF
